:020000040800F2
:10000000F00F00203D010008452C00086B29000876
:1000100000000000000000000000000000000000E0
:10002000000000000000000000000000492C000853
:100030000000000000000000472C00084D2C0008C4
:100040004F010008000000004F0100084F010008A8
:100050004F0100084F0100084F0100084F01000840
:10006000000000004F0100084F0100084F01000888
:100070004F0100084F0100084F0100080000000078
:100080004F0100084F010008000000004F01000868
:100090004F0100084F0100084F0100084F01000800
:1000A0004F0100084F0100084F01000849340008C3
:1000B0005934000800F002F800F030F80CA030C805
:1000C000083824182D18A246671EAB4654465D46D4
:1000D000AC4201D100F022F87E460F3E0FCCB6466E
:1000E0000126334200D0FB1AA246AB4633431847E1
:1000F000F04F0000105000000023002400250026CF
:10010000103A01D378C1FBD8520700D330C100D5D3
:100110000B6070471FB51FBD10B510BD00F050FD3E
:100120001146FFF7F7FF03F0E9FE00F068FD03B4A6
:10013000FFF7F2FF03BC00F09DFD00000748804779
:1001400007480047FEE7FEE7FEE7FEE7FEE7FEE7BB
:1001500004480549054A064B70470000CF2C0008AB
:10016000B5000008F0090020F00F0020F00B00207F
:10017000F00B002010B5202A04DB0846203AD040BE
:10018000002110BD0B462024D340D040A21A91403C
:100190000843194610BDFEB5054610460C461843E7
:1001A00073D0AE468C460020AD1A01469C4167D301
:1001B0006646002701243D46B61A9D4102D31346E8
:1001C0003A462124654676462F04360C3E432D0CD4
:1001D000B61A9D4104D3150C1B042B431204103492
:1001E000654676462F06360A3E432D0AB61A9D41CD
:1001F00004D3150E1B022B431202083465467646C3
:100200002F0736093E432D09B61A9D4104D3150F19
:100210001B012B431201241D65467646AF07B60825
:100220003E43AD08B61A9D4104D3950F9B002B4366
:100230009200A41C65467646EF0776083E436D089B
:10024000B61A9D411AD392185B41641C16E000183F
:10025000764665464941B71A9D410191009009D300
:100260006046B11A98418E4684460098019900254F
:10027000401C6941DD0752082A435B08641EE6D52D
:100280007246634603B0F0BDFFE700200146C0465A
:10029000C0462A462346F5E701E004C0091F0429A9
:1002A000FBD28B0701D50280801CC90700D00270E9
:1002B000704700290BD0C30702D00270401C491EB2
:1002C000022904D3830702D50280801C891EE3E73C
:1002D0000022EEE70022DFE7002203098B422CD345
:1002E000030A8B4211D300239C464EE003460B4386
:1002F0003CD4002243088B4231D303098B421CD3E8
:10030000030A8B4201D394463FE0C3098B4201D3D9
:10031000CB01C01A524183098B4201D38B01C01A11
:10032000524143098B4201D34B01C01A5241030988
:100330008B4201D30B01C01A5241C3088B4201D337
:10034000CB00C01A524183088B4201D38B00C01AE4
:10035000524143088B4201D34B00C01A5241411A0B
:1003600000D201465241104670475DE0CA0F00D0EE
:100370004942031000D34042534000229C460309E7
:100380008B422DD3030A8B4212D3FC22890112BA6D
:10039000030A8B420CD3890192118B4208D3890145
:1003A00092118B4204D389013AD0921100E089095D
:1003B000C3098B4201D3CB01C01A524183098B423E
:1003C00001D38B01C01A524143098B4201D34B0127
:1003D000C01A524103098B4201D30B01C01A52418A
:1003E000C3088B4201D3CB00C01A524183088B4211
:1003F00001D38B00C01A5241D9D243088B4201D39A
:100400004B00C01A5241411A00D201466346524184
:100410005B10104601D34042002B00D54942704783
:1004200063465B1000D3404201B50020C046C04681
:1004300002BD704770477047F0B50C46871A9C4163
:100440000D46861A9D4103D2C01BA141D2196341BA
:100450000D0D1F0DC94EEC1BAE435CD07F057F0D0B
:100460000026002F51D02D05AC46A943DD02012303
:10047000ED0A1B051D4320231B1B24D41746E74010
:10048000381871412F46E740CC199D402818314655
:1004900061410C0D27D161449A4013D50023401CC3
:1004A000594152000ED14008400001224B00520534
:1004B000D34207D305204007C14201D5B04900E02F
:1004C000B0493046F0BD6B00002A00D001229A18D6
:1004D0001F23203C1B1B01D5002302E0E540281808
:1004E00071410C0DD7D0012424050919C407CD078B
:1004F00040084908E40F28436144002CD5D000246B
:10050000401C61419A40D0D1CDE76A05520DD9D146
:10051000C90FC907D5E79C4D4E00002801D0012422
:1005200000E0002434195F00002A01D0012600E019
:100530000026BE19954FAC420CD8AE420AD8B44240
:1005400006D001256D05EC42BCD010461946F0BD21
:100550009942FCD000203946F0BDF0B51FB40C46DE
:100560000F46811A9F412546861A9D4106D20125D4
:10057000ED076F40401ABC4152187B41210D1E0D02
:100580008D1BAC467D4D8D437ED075056D0D7CD0A9
:100590000D05AE46AC431B031B0B794D52429D41EA
:1005A000202366469B1B14D31746F74038180026B5
:1005B0000090744160462F460741E41900989D4021
:1005C0002818664116D4714671189A4025D5012322
:1005D00020E093182A466A415200002B00D0521C9A
:1005E0001E23203E9B1B002B61DD3541EE17281892
:1005F0006641E8D5001876415B1C9A4000D3401C48
:100600004B05F3181524E34010D3002B52D071464C
:100610007118D30FC01802D3491C05B0F0BD0123D7
:10062000DB079A42F9D140084000F6E70122520563
:10063000B21801D1002853D00123CC0ADB02994320
:10064000891E002A08D1020C03D0020C00041039C4
:1006500002E00246002020390023550B05D112028A
:100660000823550B01D152010D23550C01D1120164
:100670001B1DD50C01D192009B1C150D01D1520000
:100680005B1C2025EE1A01E02CE022E00546F54037
:1006900015439840CA1AE10769181305C918002ABA
:1006A000BBDA032040070818C10FC9070FE07146E5
:1006B0006118B2E7F10740080843711071444A001D
:1006C0000CD001235B059A42A7D2C90FC9070020AD
:1006D000A3E74905490D26D1002001E00028F4D107
:1006E00000219AE7284D6600002801D0012100E092
:1006F000002171185F00002A01D0012600E00026C9
:10070000BE19224FA94210D8AE420ED8B14208D02D
:1007100001256D05E94206D01946A8024140104660
:100720007BE79C4201D0214677E70020394674E7F9
:1007300010B50C465C4005D50124E4076340FFF783
:100740000CFF10BDFFF778FE10BD30B40C465C40C6
:1007500004D50124E407634030BC6DE630BCFCE600
:1007600070B50124E40761400D465D4002D4FFF7F7
:1007700063FE70BD6340FFF7F0FE70BDFF07000031
:100780000000F0FF0000F07F0000E0FF0000F87FB5
:100790001F22030C02D10F22000402D0030E03D04B
:1007A00004E00020014670470002083A030F01D11F
:1007B0000001121F830F01D18000921E002801DB6F
:1007C0004000521E120551184205C0124118104631
:1007D0007047C10FC90700D0404201229207114360
:1007E000D6E701218907D3E70121C9050123411873
:1007F00042001B06D3185B0E0AD0C1100722D20696
:10080000891840075242D14201D5520089187047D9
:10081000090208D50146002A03D0C10FC9070020EC
:10082000704710467047420202D0002002497047CC
:10083000072109050143F4E70000F87FF0B5FF2523
:100840002D04C609C209FF2704462E400137CB09F3
:100850003E4348402A402B400746002A6BD0002BDD
:1008600069D0AA4267D0AB4265D0002800DA324690
:100870000125ED0529432C4309022002090AD21A59
:100880004B0C7F24E31A434C000A7C44E35C7D2438
:100890002404121914145B00A218884201D3521CBC
:1008A00000E0400049420C465C4324115C43DB01FC
:1008B0006415E318040A5C43C502200D0C4644434A
:1008C0006419250A5D432303EC0C0D4665430003C0
:1008D0000019EB184C42A34201D35B18401CD4050D
:1008E0002018002B07D05B00C91804D3401C002936
:1008F00001D1400840003F2189048A4209D3002ADF
:1009000008DC1106090F04D0032149074018C00F65
:10091000C007F0BD01224100120689187F2252064D
:100920009142F6D205214907C84201D59010F0BD89
:10093000FF20C005F0BD002F00DA32461648AA425B
:1009400007D2AB4205D21902090E17D0F80FC00723
:10095000F0BDFF2563002D06AB42F9D84900A9423E
:10096000F6D8AB4201D1A942F2D0A94201D100216F
:1009700001E061004908D0050843F0BD1102090EED
:10098000FBD0FF200243D005F0BD0A4601461046C9
:1009900054E70000124800000000C07F10B5014677
:1009A0009E240002CA15A307002A02D01843002A79
:1009B00004DBA21A002A0CDDD04010BD1206120E74
:1009C00001D140004008A21A03D4D0404042002880
:1009D000F3DDFF2248001206904201D9002010BD2D
:1009E000C817C043584010BD0102C21504D00123EE
:1009F000DB071943002A0ADB9E239A1A02D4084611
:100A0000D0407047FF2241001206914201D90020D8
:100A10007047C017C04370471F22030C02D10F223A
:100A200000041CD0030E01D10002083A030F01D1CB
:100A30000001121F830F01D18000921E002801DBEC
:100A40004000521ED205511802125118192290402E
:100A500004D3491C002801D14908490008467047C1
:100A6000C10FC90700D04042012292071143D3E7CA
:100A700001218907D0E70000F8B5224C4E00069D01
:100A8000A6420AD8A64201D1002806D15E00A6429D
:100A900003D8A6420AD1002A08D00D2424042542F6
:100AA0002CD02946002000F061F8F8BD0C461C430C
:100AB0000CD4994202D0EFF30080F8BD904202D0EE
:100AC000EFF30080F8BDEFF30080F8BD09242407A0
:100AD000E5008B4206D0EFF30080A043591A06D2FE
:100AE000284304E0101A05D3EFF30080A04380F3FD
:100AF0000088F8BDEFF30080A043F1E7009500F017
:100B00004DF8F8BD0000E0FF10B5FF231B064400C0
:100B10009C421DD84C009C421AD80346124A0B43F3
:100B200007D4401A02D3EFF3008010BDEFF300802A
:100B300010BD081A06D2EFF3008001219043C907C7
:100B4000084302E0EFF30080904380F3008810BD7B
:100B50000D231B041A4204D01146002000F006F8B1
:100B600010BD00F025F810BD00000090C80212D59D
:100B70004803400F002804D0C803C0430121884027
:100B80007047EFF3008000010009032109070843C3
:100B900080F30088704700207047000010B50020E7
:100BA0000249029A00F033F810BD00000000F87FFF
:100BB00010B5024800F02BF810BD00000000C07F07
:100BC000754600F053F8AE46050069465346C00826
:100BD000C000854618B020B5FFF7BAFA60BC002700
:100BE0004908B6460026C0C5C0C5C0C5C0C5C0C5F9
:100BF000C0C5C0C5C0C5403D49008D46704710B551
:100C00000446C046C0462046FFF791FA10BD10B515
:100C10000C461107090F092904D00A290AD008290E
:100C20000CD104E011460820FFF7A0FF06E05106B2
:100C300006D501E0510601D50120C007214610BDAF
:100C4000D10607D501010909CC084907000E0006A5
:100C5000044309E0410F20024907000A0143200E26
:100C600000061D22D14101430846E7E700487047CE
:100C70009009002001491820ABBEFEE726000200C3
:100C8000704770B58C180578401C6B075B0F01D15D
:100C90000378401C2A1106D10278401C03E0067834
:100CA000401C0E70491C5B1EF9D12B0705D4002394
:100CB000521E0DD40B70491CFAE70378401CCB1A66
:100CC000921C03E01D780D70491C5B1C521EF9D567
:100CD000A142D8D3002070BD10B50146406A826B96
:100CE00050231A420AD1816B0122520211438163BF
:100CF0000168CA681205920F05D020E0006B026BF4
:100D00000846904710BD827E002A18D10A68120753
:100D100015D58A6853070122002B09DB4B680C2488
:100D2000A3434B60816B130299431143816306E037
:100D3000816B202319438163C16B1143C16300F0B0
:100D4000A5FB10BD10B5406A816B40221143816341
:100D5000C16B04221143C16300F09AFB10BD10B5B2
:100D6000406A00F094FB10BDF8B5044600200090E6
:100D7000206881688907890F012905D10168C907A1
:100D80002CD1C168090429D48168154A1026114064
:100D90000125002915D18168294381601248114934
:100DA0000068FFF799FA00E0401E00900028FBD190
:100DB00000F0B0FE07460CE000F0ACFEC01B0228BD
:100DC00007D9A06B3043A063E06B2843E0630120A8
:100DD000F8BD20680068C043C007EDD10020F8BD11
:100DE0001700008040420F000C05002010B504469B
:100DF0000068054940181421FFF76EFA800020644E
:100E00000248E06310BD0000F8FFFDBF0000024093
:100E100030B5056C0124AC40C56B6C600468636040
:100E20004368102B036803D099600068C26030BD2E
:100E30009A600068C16030BD0E490A880E49098871
:100E400000280DD0012813D10C48002902D0002A17
:100E500003D009E082420BD008E0814206D007E0CF
:100E6000002A05D0002901D0AB207047012070472F
:100E70000020704700780008007C0008EEEE0000BB
:100E80001FB50020134C03900090012120460194CF
:100E9000029100F081F9002805D103A9684600F00D
:100EA000E1FC002814D1002213462146012000F065
:100EB00029FD00280CD10848019000F06DF90028A8
:100EC00005D103A9684600F0CDFC002800D1002020
:100ED00004B010BD00780008007C0008F0B585B0B3
:100EE0000024574E03943288671E564D28880121EE
:100EF0000291390C01960094002A68D0524BD21806
:100F000021D05249CA421BD1002808D059428842F8
:100F100016D1304600F040F9002807D00CE03046EA
:100F200087E003A9684600F09DFC4BE003A96846F2
:100F300000F098FC002848D10022134629463EE0E4
:100F4000FFF79EFF3EE0002808D08842F8D12846EF
:100F5000019500F021F9002828D02DE03848C288FA
:100F60003B496600885B824200D127B2BC420ED06A
:100F70003749891E00F0C4F8012808D034493448A4
:100F8000891E805B098800F0DDF800281DD1641CF3
:100F9000A4B2042CE2D3002213462949012000F018
:100FA000B1FC002811D1009028463FE003A9684613
:100FB00000F058FC002808D10022134631460120D9
:100FC00000F0A0FC002800D1002005B0F0BD0028F2
:100FD000B6D0884202D1284601952AE01948C18836
:100FE0001B486500425B914200D127B2BC420FD042
:100FF00017491046891E00F083F8012808D01449CB
:101000001348891E405B098800F09CF80028DCD159
:10101000641CA4B2042CE1D3002213460949012028
:1010200000F070FC0028D0D10090304601210291E0
:10103000019000F0B1F8002800D172E7C4E7000089
:1010400000780008007C00081211FFFFEFEEFFFFA0
:1010500002000020F3B5264C002685B00F46254639
:1010600030460396FFF7E8FE2249012804D0002805
:1010700004D0AB2007B0F0BD0C4600E00D461E4A80
:1010800000232946012000F03DFC0028F2D139461A
:10109000059800F057F80028ECD118497700C85B94
:1010A000059A90420DD0891E00F02AF8012808D038
:1010B00012491248891EC05B098800F043F80028D5
:1010C000D8D1761CB6B2042EE7D3002000900120C0
:1010D0000290019403A9684600F0C4FB0028C9D11E
:1010E000002213462946012000F00CFCC2E7000054
:1010F00000780008007C0008EEEE000002000020EE
:10110000F8B506460D4601240C4F0020FFF794FE6B
:10111000AB2811D081020A4AC8198A18801C08E03D
:101120001188B14204D1403AD08F2880002402E0D7
:10113000121F8242F4D82046F8BD00000078000853
:10114000FE7B000870B506460D46114C0120FFF7E6
:1011500073FEAB280BD080020E490419401803E03F
:101160002168491C04D0241D8442F9D3802070BD1D
:101170002A4600232146012000F0C4FB0028F6D1B6
:1011800032460023A11C012000F0BCFB70BD000012
:1011900000780008FF7B000810B50121064B074CC2
:1011A00005E002889A4201D0002102E0001DA04221
:1011B000F7D9084610BD0000FFFF0000FF7B0008C4
:1011C00070B50C460546FFF7BDFF802803D12146C8
:1011D0002846FFF73FFF70BD72B6FEE706490020C4
:1011E000C861064801690422114301610169402276
:1011F0001143016170470000700900200020024087
:10120000064A0021D16106490A6902231A430A618C
:101210004861086940221043086170477009002046
:101220000020024010B5054B0022DA61044A136920
:10123000012423431361018010BD000070090020C8
:101240000020024010B50B4A0020D168CB060A49A5
:1012500004D5C86902231843C8611020D3685B070E
:1012600005D5CB6901242343CB6104210843D06019
:1012700010BD0000002002407009002070B5054636
:1012800000F048FC0646104C0AE0681C08D0002D0F
:1012900004D000F03FFC801BA84201D9032070BDA0
:1012A000E068C007F1D1E068800601D52020E06049
:1012B000E068C00602D4E068400703D5FFF7C2FF2C
:1012C000012070BD002070BD00200240F8B5054629
:1012D00004462035287D0026012808D001202875E5
:1012E000206881688907890F012908D101E002205F
:1012F000F8BD0168C90738D1C168090435D4A16BAC
:10130000FF220132914302221143A163C168890780
:10131000890F0091C16889088900C16020688168CF
:1013200092071143816000F0F5FB07460EE000F0E4
:10133000F1FBC01B022809D9A06B022188431021B0
:101340000843A063002028750120F8BD206880684C
:101350000028ECDB2068C168009A1143C160A06BD3
:1013600080088000401CA06304E0A06B202108439B
:10137000A0630126002028753046F8BDF8B5002589
:10138000044620340095227D012A39D0012222759D
:1013900003689E68760767D4384F4E68BE424DD0CA
:1013A0009E6A0F78BA4016439E620123C26A1B07E9
:1013B0009A421FD0012A1DD0022A1BD0032A19D01D
:1013C000042A17D0052A15D0062A13D0072A11D0CF
:1013D00002688B6856697607760FB3420AD0536964
:1013E000DB08DB005361006842690B7A5B075B0F27
:1013F0001A4342610A68102A04D0112A02D038E048
:101400000220F8BD1E488368102A07D001229205E9
:10141000134383600868102803D02AE00122D20514
:10142000F6E7194817490068FEF756FF0A214843B6
:1014300000E0401E00900028FBD11AE0986A0E7868
:10144000B240904398620968102901D0112910D147
:101450000B488268102904D0012189058A438260E3
:1014600007E00121C905F9E7816B2022114381635F
:101470000125002020752846F8BD0000011000005D
:101480000027014040420F000C05002070477047C4
:1014900070470000F8B500260446002805D0A06B70
:1014A00025462035002802D007E00120F8BD0020A5
:1014B000E0632875204600F0A9F8A06B1022C00652
:1014C000002870DB2068816849076CD4A16B130188
:1014D000994302231943A16381688907890F012970
:1014E00005D10168C9070FD1C16809040CD4C168CE
:1014F00018239943A3681943C16020680169636890
:1015000089008908194301612068C1683D4B194071
:10151000C160207E617E8003C9030843A17E4B0326
:101520001843A36A012B02D001231B0300E0002310
:101530001843E36818432369022B09D0002318439A
:101540002B79E57E5B0018430123012D02D00AE0D0
:101550000423F4E7002927D0A16B20252943A163A8
:10156000E16B1943E163E1690D46FF3DC23D02D0E5
:10157000256A294308432168CD680543CD600125CC
:10158000E16A2D07A94213D0012911D002290FD0F9
:1015900003290DD004290BD0052909D0062907D02D
:1015A000072905D010E028E0012109040843DAE703
:1015B00021684D69ED08ED004D6121684D69A78DE9
:1015C0007F077F0F3D434D612168C9680E4D29405B
:1015D000814207D10020E063A06B80088000401C9E
:1015E000A06308E0A06B022188431043A063E06B76
:1015F0001843E06301263046F8BDA06B1043A0639A
:10160000F8E700001902FEFFE7FF3F83F0B587B05F
:10161000054614216846FEF75DFE1B49286888428E
:101620002FD11A4988694E15304388618869304046
:1016300005904A69300202434A6149690027014026
:1016400005917020009003200190092069460297BF
:10165000C00600F0A9F90E480E4C81C42760802016
:10166000A66060600001E060202067612061094899
:10167000083C00F085F8002801D0FFF7ADFD2C6391
:10168000656207B0F0BD0000002401400010024078
:1016900008000240EC070020F7B50446006800256A
:1016A000806840073DD426462036307D01280AD088
:1016B00001273775607E012807D02046FFF754FBCD
:1016C000050002D02EE00220FEBDA06B16490840A6
:1016D000FF2101310843A0630020E0633075216BD6
:1016E00012488862216B1248C862216B1148086356
:1016F00021681C2008602068416810221143416065
:101700002068C1683943C1602168206B4031029B69
:10171000019A00F05FF8206881680422114381601B
:1017200000E002252846FEBDFEF1FFFFD90C0008AF
:101730005F0D0008450D000870B5002401462031FA
:101740004A78022A03D004218163012416E002684A
:1017500013680E25AB431360026813685B085B00D7
:1017600013600122056C1346AB40C56B6B604A7079
:1017700000220A70416B002900D08847204670BDC6
:1017800070B5040021D0022120462030054641706A
:10179000226811680E48A3680140606826691843F2
:1017A000E3683343184363691843A3691843E36943
:1017B0001843084310602046FFF718FB0021A1637F
:1017C000012068702970084670BD012070BD0000BE
:1017D0000FC0FFFFF8B504468C4620300178002585
:1017E000012909D00126067041780027012905D07A
:1017F000077002252846F8BD0220F8BD022141707D
:10180000A7632068016849084900016061462046D5
:10181000FFF7FEFAE06A00282068016802D00E2275
:10182000114306E00A221143016020680168042286
:10183000914301602068016831430160DAE70000EC
:1018400070B5044600F066F90546601C02D00448F5
:101850000078241800F05EF9401BA042FAD370BD56
:1018600000050020F8B5054623480F46017E0126F5
:1018700001290BD0012101762868204C012807D0CE
:101880002046FFF7FBFC002813D030E00220F8BD13
:101890002046FFF7F3FC002829D1FFF79FFC2046E4
:1018A000FFF7ECFC064616480169042291430161EA
:1018B0001DE00020C04338606C6812E02046FFF74E
:1018C0009FFC0E48FFF7DAFC06460D48026902212C
:1018D0008A430261002E01D03C6008E001208002B2
:1018E0002418A868810268680818A042E6D802484F
:1018F000002101763046F8BD7009002050C3000079
:1019000000200240F0B51FB407461A480024017EAB
:1019100015461E46012907D0012101761648FFF71A
:10192000ADFC002803D020E0022005B0F0BD012F5F
:1019300002D0022F00D00427220128463146FEF7AC
:1019400019FC81B2019862001018FFF76BFC0A487D
:10195000FFF794FC09490A69520852000A610028FD
:1019600003D1641CE4B2BC42E6D3024900220A76E9
:10197000DBE700007009002050C300000020024097
:10198000064900200A69120607D5054A4A60054A39
:101990004A600969090600D501207047002002400D
:1019A00023016745AB89EFCDF8B500238DE0012415
:1019B0009C40A44622407DD04C68022C01D0122CC1
:1019C0000CD1DC08A40027183C6A5D07ED0E0F2639
:1019D000AE40B4430E69AE4026433E6205685E00E9
:1019E0000324B4400F79A543BF07BF0FB7402F436F
:1019F00007604D68012D05D0022D03D0112D01D0B7
:101A0000122D0ED18568CF68A543B7402F4387605C
:101A100047686546AF430D79ED06ED0F9D403D43A8
:101A20004560C568A5438C68B4402C43C4604C68CD
:101A3000E40049D5284CA56901263543A561A46970
:101A40009D0834400094254CAD002F19BC689D07BB
:101A50002E0F0F25B540AC430925ED06A84201D154
:101A600000250FE01E4DA84201D101250AE01D4DC1
:101A7000A84201D1022505E01B4DA84201D1032552
:101A800000E00525B5402543BD60184C25684E682B
:101A90009543F60300D51543256065684E68954368
:101AA000B60300D515436560A5684E689543F602F8
:101AB00002D500E008E01543A560E5684E6895434F
:101AC000B60200D51543E5605B1C0A681446DC408D
:101AD00000D06CE7F8BD000000100240000001409B
:101AE0000004004800080048000C004800040140C1
:101AF0000069084000D00120704742690A4200D0C6
:101B0000090481617047002A01D0816170478162B8
:101B10007047000001488068704700000005002001
:101B200002488168027889188160704700050020AA
:101B300010B506480168102211430160032000F02F
:101B400007F800F027F8002010BD00000020024038
:101B500070B504460D4D7D202978C000FEF7BCFB12
:101B600001460B480068FEF7B7FB00F043FB002876
:101B700009D1042C07D200222146401E00F02AF889
:101B800000206C6070BD012070BD000000050020C9
:101B90000C05002008B508488169012211438161C4
:101BA000816911400091C26901040A43C261C069A0
:101BB0000840009008BD000000100240002805DB2E
:101BC000C106C90E01208840014908607047000025
:101BD00000E100E010B501F06DFC10BDF8B5054660
:101BE0000068354CC00352D5E0690026C00007D418
:101BF000E16920040143E161E169014001260091AE
:101C00002E480168C90510D401688215114301608E
:101C1000FFF780FF074604E0FFF77CFFC01B642846
:101C200024D826480068C005F6D5206A03273F025D
:101C3000384020D06968394081421CD0206A226A2D
:101C4000B843012109040A432262226A8A432262BC
:101C50002062C0070FD0FFF75DFF009008E0FFF79C
:101C600059FF0099411A1648814201D90320F8BD55
:101C7000206A8007F3D5206A6968B8430843206268
:101C8000002E04D0E169012000078143E16128783A
:101C9000C00705D0206BA968800880000843206336
:101CA0002878800605D5206B10218843E968084311
:101CB00020630020F8BD00000010024000700040CA
:101CC00088130000F8B50F46060059D03A4D286831
:101CD000C007C00FB84209D2286840084000384306
:101CE00028602868C007C00FB84249D13068334C1B
:101CF00081070CD5400704D5606807210902084315
:101D000060606068F0218843B168084360603078A3
:101D1000C00726D0706801280ED0216802280ED096
:101D2000890700292CDA616889088900014361600C
:101D3000FFF7F0FE00900DE021688903F1E78901CB
:101D4000EFE7FFF7E7FE0099411A1D48814201D9EC
:101D50000320F8BD60680C21084071688900884242
:101D6000EFD12868C007C00FB8420BD928684008D7
:101D70004000384328602868C007C00FB84201D02F
:101D80000120F8BD3078400706D5606807210902B8
:101D90008843F1680843606000F028F86168094AE8
:101DA0000906090F515CC840074908600320FFF786
:101DB000CFFE0020F8BD00000020024000100240CD
:101DC00088130000885000080C05002004480549CD
:101DD00000684968044A4905490F515CC84070478A
:101DE0000C050020001002409850000810B514A304
:101DF0000FCB88B06C460FC415A30FCB0FC4184A85
:101E000051680C200B4603401648042B16D0082BB3
:101E100014D18B021B0F6C46E45CD26A04AB120730
:101E2000120F9A5CC90305D500231946FEF7B3F9D2
:101E3000214601E020460C4901F016FB08B010BD18
:101E400002030405060708090A0B0C0D0E0F1010FB
:101E50000102030405060708090A0B0C0D0E0F10FA
:101E60000010024000127A0000093D00FEB5040097
:101E700070D02078DC4DC0074AD068680007800F1A
:101E8000012807D068680007800F022809D1686818
:101E9000C00306D5286880033AD560680028E7D0DB
:101EA00036E06168012914D001208004002901D0A6
:101EB000052914D02A68012109048A432A60296867
:101EC000814329606068002816D0FFF723FE06468C
:101ED0000EE028680121090408432860F2E7296818
:101EE00001432960F5E7FFF715FE801B64286ED8D3
:101EF00028688003F7D50BE0FFF70CFE064604E0E8
:101F0000FFF708FE801B6428F1D828688003F7D407
:101F100020780126800700283CDA68680007800FD7
:101F200007D068680007800F022809D16868C003DD
:101F300006D42868800716D5E06801280AD112E087
:101F4000E0680028286816D030432860FFF7E2FDDB
:101F5000074605E043E1FFF7DDFDC01B0228C6D8B8
:101F600028688007F7D52868F82188432169C900C7
:101F7000084328600EE0400840002860FFF7CAFDD3
:101F8000074604E0FFF7C6FDC01B0228AFD828684B
:101F90008007F7D42078000722D5E0690028686A16
:101FA0000ED030436862FFF7B5FD074604E0FFF747
:101FB000B1FDC01B02289AD8686A8007F7D50FE0E8
:101FC000400840006862FFF7A5FD074605E09DE078
:101FD000FFF7A0FDC01B022889D8686A8007F7D4E4
:101FE000207804274007002860DA00200190E86983
:101FF000C00008D4E969B8060143E961E969014014
:1020000001200091019079480168C90511D4016847
:10201000821511430160FFF77DFD009005E0FFF799
:1020200079FD0099401A642870D870480068C0058E
:10203000F5D5A06801280AD0002801D0052810D0C5
:10204000286A400840002862286AB84301E0286AEC
:1020500030432862A068002812D0FFF75BFD009093
:102060000AE0286A38432862F1E7FFF753FD009938
:10207000411A5F48814249D8286A8007F5D50DE0AA
:10208000FFF748FD009006E0FFF744FD0099411A74
:10209000574881423AD8286A8007F5D40198002829
:1020A00004D0E969012000078143E9612078C00676
:1020B00035D5606901280CD0401D686B23D03843AA
:1020C0006863686B400840006863FFF723FD0646BD
:1020D00022E0686B38436863686B30436863FFF7DE
:1020E00019FD064604E0FFF715FD801B02285BD8AA
:1020F000686B8007F7D5686BF8218843A169C90030
:10210000084368630BE0B8436863F4E74CE0FFF70B
:1021100001FD801B022847D8686B8007F7D4206A2E
:1021200000285ED069680907890F022942D001267C
:1021300036060228286805D0B0432860FFF7EAFC7D
:10214000044633E0B0432860FFF7E4FC074604E0B0
:10215000FFF7E0FCC01B022826D828688001F7D4CE
:10216000E86AE16A000900010843E862616AA06A5E
:10217000084369683D221204914308436860286857
:1021800030432860FFF7C6FC044604E0FFF7C2FCBA
:10219000001B022808D828688001F7D521E0FFF746
:1021A000B9FC001B022801D90320FEBD286880016C
:1021B000F5D416E00128F8D06868E96A0122120413
:1021C000636A02409A420AD10907E26A090F914202
:1021D00005D10F2189040840A16A884201D001205D
:1021E000FEBD0020FEBD0000001002400070004057
:1021F00088130000094910B5401E884201D901200A
:1022000010BD074C60610321081F01F053F9002045
:10221000A06107202061002010BD0000FFFFFF002B
:1022200000E000E030B5034620331A7F012A26D0B3
:1022300001221A770325CA682D02AA438D6800245B
:102240002A430125AD02AA434D6800682A430125AF
:10225000ED02AA430D682A4301252D03AA430D6907
:102260002A4301256D03AA434D69C9692A43012503
:10227000AD03AA430A4342641C77002030BD02200C
:1022800030BD0000F0B502462032137F012B1ED076
:10229000012515770223537706687468B3687027A1
:1022A000BC430F682743776000680A4CA04205D002
:1022B000094CA04202D0094CA04204D180244968B4
:1022C000A34319438160557700201077F0BD0220A9
:1022D000F0BD0000002C014000040040004001401F
:1022E00010B504460068042200F036FD2068416CF9
:1022F0000122D20311434164206881684907490FD4
:10230000062903D00168012211430160002010BD9D
:1023100070B5040005D025462035687F002802D01E
:1023200006E0012070BD00202877204600F00AF862
:1023300002206877211D206800F0CAFC0120687720
:10234000002070BD08B500680549884207D10548DE
:102350008269C1140A43826180690840009008BD07
:10236000002C014000100240F8B505460446203517
:10237000287F012817D001262E770220687722684F
:1023800090687727FF23B8431B02984390600A6840
:10239000502A31D00EDC202A4BD006DC002A48D04F
:1023A000102A3AD145E00220F8BD302A41D0402A17
:1023B00033D136E0602A27D0702A12D001200003E2
:1023C000121A2AD0824228D1CB684A6889682068CC
:1023D00000F0CFFC206881680122920311438160E4
:1023E0001BE0CB684A688968206800F0C2FC21685D
:1023F00088683843886010E0CA684968206800F03F
:10240000C7FD5021206806E0CA684968206800F0CE
:10241000D0FD6021206800F0B7FC6E77002028779F
:10242000F8BDCA684968206800F0B2FD4021206804
:10243000F1E711462068EEE710B586B00446142196
:102440006846FDF747FF0D492068884214D10C48C3
:102450004269012189040A434261406908400590AC
:102460000811009002210020019102900491039034
:1024700069460448FFF798FA06B010BD002C0140E9
:102480000010024000040048F8B506460446203615
:10249000307F0D4601280DD0012030770220707763
:1024A0000427002A08D0042A16D0082A2AD00C2A89
:1024B0004DD137E00220F8BD206800F06DFC2068A7
:1024C000816908221143816120688169B943816172
:1024D000206881692A6912E0206800F0A1FC206868
:1024E00082690121C9020A4382612068816901224F
:1024F000920291438161206881692A691202114325
:10250000816124E0206800F0CBFC2068C2690821CA
:102510000A43C2612068C169B943C1612068C169C9
:102520002A6912E0206800F0FDFC2068C1690122E0
:10253000D2021143C1612068C269012189028A4324
:10254000C2612068C1692A6912021143C161012078
:10255000707700203077F8BD70B5040005D02546AF
:102560002035687F002802D006E0012070BD0020E1
:102570002877204600F00AF802206877211D20689D
:1025800000F0A6FB01206877002070BD70477047FF
:10259000F8B502680446D069116893684C4D064648
:1025A0002E402025002E68D0DE07F60FFF272137AA
:1025B0000F40374375D0C70706D0CF0504D5012794
:1025C0001762E26F3A43E267820708D5DA0706D05E
:1025D000276802223A62E26F04273A43E267420721
:1025E00008D5DA0706D0236804221A62E26F0223B4
:1025F0001A43E267020709D50A462A40324305D04A
:10260000236808221A62E36F1343E367020508D5C3
:102610004A0106D501222368D2021A62E26F2A43D8
:10262000E267E26F002A30D0800606D5880604D51E
:10263000216E002901D020468847E06F2168896813
:10264000490602D42821084224D0204600F064FD27
:1026500020688168490619D58168402291438160CC
:10266000E06E002812D01B494163E06EFFF764F86A
:1026700000280AD0E06E416B06E0830611D58B0678
:102680000FD5216E12E020468847F8BD2046FFF79F
:102690007EFFF8BD2046FFF77AFF0020E067F8BD17
:1026A000FFE7030605D50B0603D5616E0029EAD1C5
:1026B000F5E74006F3D54806F1D5116820464023DA
:1026C0009943116065670021616600F04DF9E6E706
:1026D0000F0800000531000810B5040003D0606F3A
:1026E000002802D007E0012010BD00217020015514
:1026F000204600F027F82420606720680168490818
:1027000049000160204600F06FFD0128ECD0606AAE
:10271000002802D0204600F05FFC206841680122BA
:10272000D202914341602068816808229143816010
:1027300020680168012211430160204600F0B2FCCC
:1027400010BD0000F0B587B0044614216846FDF7BF
:10275000C1FD264F01212668002225484904022395
:1027600003240125BE421DD18769CE1037438761FE
:1027700087693740059746690E4346614069019372
:10278000084005906002009002AE34C609206946F8
:10279000C006FFF709F9002211461B20FFF71AFABD
:1027A0001B201EE0134FBE421DD1C6690E43C661F9
:1027B000C6690E40059646690E434661406901931D
:1027C000084005900C20009002AE34C609206946EE
:1027D000C006FFF7E9F8002211461C20FFF7FAF9BE
:1027E0001C20FFF7EBF907B0F0BD000000380140F6
:1027F0000010024000440040F0B5836F202B49D107
:1028000000290AD0002A08D08568DC01A54206D13B
:102810000369002B03D1CB0701D00120F0BD034693
:1028200060331E7C012E35D001271F74416501469F
:1028300040310A834A830022FF260266A54204D162
:102840000569002D22D1144D1EE0002D18D08A8379
:10285000C2672221816701688D683D438D60816870
:10286000A14202D10169002912D00C4901661A74F3
:1028700000680168FF222132114301600020F0BD91
:102880000569002D02D07F258D83E1E78E83DFE788
:102890000349EBE70220F0BDFF0100009131000881
:1028A0003931000870B5044600680C4901260C4D0A
:1028B000884206D12946AE76012232310948FFF717
:1028C0009BFF09492068884206D10549EE7601221E
:1028D00031310648FFF790FF70BD0000003801401D
:1028E0000C0000207008002000440040F008002088
:1028F00070B5436F202B30D100290AD0002A08D0B0
:102900008568DC01A54206D10369002B03D1CB0702
:1029100001D0012070BD034660331E7C012E1CD007
:1029200001261E74C164014640310A824A82002198
:102930004166C16721224267A54202D10269002A8D
:1029400009D0074A42661974006801688022114361
:102950000160002070BD034AF4E7022070BD000052
:1029600071330008313300087047FEE73EB500219F
:1029700021480091019102911E4A41600260034684
:102980008160012204240C3316C3017641768276DD
:10299000FF23C176C233C3610162014620310A714F
:1029A0008262FEF777FD002801D0FEF715FC0120BA
:1029B0000003019007200290009469460E48FEF73C
:1029C000DDFC002801D0FEF707FC052000906946D9
:1029D0000948FEF7D3FC002801D0FEF7FDFB0620D6
:1029E000009069460448FEF7C9FC002801D0FEF7B4
:1029F000F3FB3EBD00240140AC07002008B50448AD
:102A0000416901221143416140691040009008BDB5
:102A100000100240F0B587B014216846FDF75AFC5B
:102A2000314842690121C9040A43426142690A40AE
:102A300005924269C9000A43426142690A4005920F
:102A4000426949110A43426142690A40059242695A
:102A500049000A4342614069244F08400C11059027
:102A6000002221463846FFF74EF800220121204877
:102A7000FFF749F8092000228021C006FFF743F83C
:102A80001C4E002231461C48FFF73DF800940024FC
:102A9000012501950294694638460394FEF784FFA8
:102AA000009502946946124801950394FEF77CFF55
:102AB0008020009009200294694601950394C00685
:102AC000FEF772FF029469460B4800960195039445
:102AD000FEF76AFFE80300900194694602940648F5
:102AE000FEF762FF07B0F0BD00100240000800488A
:102AF00000140048013000000004004810B596B0F2
:102B000000240F9410941194129413941C2108A87B
:102B10001494FDF7DFFB20216846FDF7DBFB2B4813
:102B2000294901600F2184604160046144612849A2
:102B30008461C160FFF7ECFB002801D0FEF74CFB7D
:102B4000012000030F900FA92048FFF70DFC00287B
:102B500001D0FEF741FB1D48FFF7FEFC002801D025
:102B6000FEF73AFB139413A918481494FFF78AFB55
:102B7000002801D0FEF730FB60200D9409940890E6
:102B80000A940B940C94042208A90E940F48FFF7A2
:102B90007BFC002801D0FEF71FFB012000944003BE
:102BA000029405900194039404946946079407489D
:102BB000FFF738FB002801D0FEF70EFB0348FFF7B4
:102BC0003BFC16B010BD0000002C01403008002076
:102BD000E703000010B50C480A4901604B21890148
:102BE000416000218160C16001618161C1610C228D
:102BF000016242614162FFF76FFD002801D0FEF7DC
:102C0000EBFA10BD003801407008002010B50C48E8
:102C10000A4901604B218901416000218160C16046
:102C200001618161C1610C22016242614162FFF771
:102C300053FD002801D0FEF7CFFA10BD004400403C
:102C4000F0080020FEE770477047000010B5FEF75F
:102C500067FF02490120087010BD0000FC0400203D
:102C600030B595B030216846FDF734FB00240125CE
:102C70000F941220059500900D940E94102010943E
:102C8000129413940C940395049006901194089454
:102C90006846FFF7EBF8002801D072B6FEE7072080
:102CA0000C900D940E9400210F940CA8FFF70AF8D5
:102CB000002801D072B6FEE710A810951294FEF716
:102CC0008DFF002801D072B6FEE715B030BD704709
:102CD000F0B502681A4B1B4C984201D0A04203D1B8
:102CE0007025AA434D682A43174D184E184F984235
:102CF0000AD0A04208D0174CA04205D0A84203D069
:102D0000B04201D0B84205D11446032212029443C6
:102D1000CA6822438024A2434C69224302608A6825
:102D2000C2620A688262984205D0A84203D0B042CB
:102D300001D0B84201D10969016301214161F0BDAF
:102D4000002C0140000400400040014000440140CC
:102D5000004801400020004010B5CB06DB0E0421E6
:102D6000046A99408C430462016A9A4011430162EB
:102D700010BD30B58468FF252D021B021343AC4300
:102D80000B432343836030BD826870239A430A4318
:102D900007210A4382607047F0B5026A5208520068
:102DA0000262056A436882697024A24392080C6833
:102DB00092001443022295438A68164E2A43144D0A
:102DC000A84207D0B04205D0134FB84202D0134FEB
:102DD000B84206D10827BA43CF6817430422974365
:102DE0003A46A84207D0B04205D00B4DA84202D0C7
:102DF0000A4DA84206D103252D02AB434D691D4360
:102E00008B692B4343608461496841630262F0BD72
:102E1000002C0140004001400044014000480140B6
:102E200070B5026A10239A430262056A4268836998
:102E300073242402A3430C6824021C4320239D43D3
:102E40008B681B012B43124DA84208D11D46CB684D
:102E50008026B5431B012B434025AB4308E00D4DB5
:102E6000A84205D00C4DA84202D00C4DA84208D172
:102E70000325AD02AA434D69AD0015438A6992004E
:102E80002A434260846149688163036270BD000027
:102E9000002C014000400140004401400048014036
:102EA00070B5026AFF2301339A430262056A4368E0
:102EB000C2697024A24392080C6892001443012254
:102EC000520295438A6812022A43124DA84208D141
:102ED0001546CA68C614B54312022A430515AA430B
:102EE00008E00D4DA84205D00C4DA84202D00C4D73
:102EF000A84208D103252D03AB434D692D011D4385
:102F00008B691B012B434360C4614968C163026242
:102F100070BD0000002C0140004001400044014011
:102F20000048014030B5026A01231B039A43026244
:102F3000046A4268C36973252D02AB430D682D02F4
:102F40001D4301235B039C438B681B0323430C4CF1
:102F5000A04208D00B4CA04205D00B4CA04202D09E
:102F60000A4CA04205D10124A403A2434C69A40148
:102F700022434260C56149680164036230BD0000BC
:102F8000002C014000400140004401400048014045
:102F900030B5036A046A6408640004628469F02539
:102FA000AC43120122430A24A3430B438261036210
:102FB00030BD30B5036A1024A34303628469036AF9
:102FC0000F252D031203AC432243A024A343090180
:102FD00019438261016230BD10B5818CC90707D0E9
:102FE00001684A6801235B049A43836A1A434A6072
:102FF000818C890707D501684A6801231B049A431D
:10300000C36A1A434A60818C490707D501684A6838
:1030100001239B049A43036B1A434A60818C09077E
:1030200007D501684A680123DB039A43436B1A43BF
:103030004A60818CC90607D50268916801231B0389
:103040009943836B19439160818C890607D5016888
:103050008A6801235B039A43C36B1A438A60818C9D
:10306000490612D503685A6801210905046C8A4390
:1030700022435A60026C8A4207D1026851680323D6
:103080005B059943436C19435160818C090607D550
:1030900001684A680123DB04806C9A4302434A605A
:1030A00010BD0000F8B500260446C667FEF732FDE5
:1030B000054620680068124F000709D501212B46FC
:1030C000002249052046009700F070F900280DD134
:1030D0002068006840070BD501212B460022890596
:1030E0002046009700F062F9002801D00320F8BDC7
:1030F00020206067A067603426740020F8BD0000BF
:10310000FFFFFF0110B5406A0022014640314A83AB
:103110004A82FFF73CFA10BD01680A68FF23213399
:103120009A430A6001688A68520852008A60202126
:10313000816700210166704710B5014640318B8BD5
:10314000846F0268222C04D09069082108439061A2
:1031500010BD928C446D1A402280426D921C4265D3
:103160004A8B521E4A83498B0029F1D101680A68B3
:10317000FF2321339A430A6001688A68520852008B
:103180008A602021816700210166FFF78BFB10BD5B
:1031900010B5014640318B8B846F0268222C04D01D
:1031A000906908210843906110BD928C1A40436DCC
:1031B0001A70426D521C42654A8B521E4A83498BDB
:1031C0000029F1D101680A68FF2321339A430A607C
:1031D00001688A68520852008A60202181670021B4
:1031E0000166FFF75FFB10BD70B50446806821697A
:1031F000E2690843616900251143226808431168A8
:10320000444B1940014311602168486803221203AE
:103210009043E26810434860A169206A226808432D
:1032200091680B231B029943014391603A4920683E
:10323000884210D13948006B8007800F11D00128D7
:1032400005D0022805D003280AD1022009E0042075
:1032500007E0082005E03249884201D1002000E063
:1032600010200122E169D2032E4E914228D100287C
:1032700006D0022807D0042817D0082844D11AE025
:10328000FEF7A4FD13E06168274A48088018FDF79F
:1032900023F880B201461039B14235D82149491C82
:1032A00001400007400F084321E0FEF79FFD6168E1
:1032B00040004A08EAE76168012248081204E5E78D
:1032C000002806D0022807D0042813D008281BD1D4
:1032D00016E0FEF77BFD0FE06168144A480811E034
:1032E000FCF7FAFF80B201461039B1420CD82168D0
:1032F000C8600AE0FEF77AFD61684A081018EFE737
:10330000616848088018EBE70125002020666066A8
:10331000284670BDF369FFFF0038014000100240ED
:1033200000440040EFFF00000024F40000127A0087
:10333000416F212910D1014640314A8A002A0CD020
:10334000C26C03681288D205D20D1A85C26C921C19
:10335000C264488A401E4882704701680A68802318
:103360009A430A6000680168402211430160704777
:10337000416F21290ED1014640314A8A002A0AD0E4
:10338000C26C036812781A85C26C521CC264488AE7
:10339000401E4882704701680A6880239A430A6089
:1033A000006801684022114301607047FFB581B099
:1033B00005460F46044660350A9E38E0701C36D03C
:1033C000FEF7A8FB0499401AB04221D8002E1FD066
:1033D0002068016849072AD5C069C043000526D482
:1033E00001202168C002086220680168FF22A13222
:1033F000914301602068816849084900816020206C
:103400006067A067E06700202874032005B0F0BD66
:1034100020680168FF22A132914301602068816821
:1034200049084900816020206067A067EBE72068B9
:10343000C1693846884305D0002103988142BDD038
:103440000020E3E70121F8E710B50248FFF7A0F8F4
:1034500010BD00007008002010B50248FFF798F872
:1034600010BD0000F0080020F8B5040C8BB2264611
:1034700082B25E430D0C1046370C58433604801957
:103480000021794116466E43370C36048019794184
:1034900026466E438919F8BD30B47446641E2578FB
:1034A000641CAB4200D21D46635D5B00E31830BC78
:1034B000184700008307FF22DB0E9A408907090E98
:1034C0009940002808DB830809489B001B181868EE
:1034D00090430843186070470007000F08388308BE
:1034E00004489B001B18D86990430843D861704773
:1034F00000E400E000ED00E0F0B52B487D22C66E50
:10350000D200761CC666016F491C0167914247DDF7
:1035100000210167406B2549864644182248244F04
:10352000803802464032158801462031AC46CB7BBC
:10353000C57DBC4204D26446022C01D1012D09D0C4
:10354000194C1C4F803C2478BE4500DD6646012B9B
:1035500027D01BE0184D144CAE421ADD0025E5665D
:10356000403C6488002B00D10470641CA4B2012389
:103570005480092C08D90C7C002C02D1447B641C9B
:1035800044730B7409245480CB7302E000220A7444
:10359000CA73417B032903D9817B102211438173B4
:1035A000F0BD5480F2E700008C000020FFFF7F4058
:1035B000FFFF9F020000404060EA0000F8B550485D
:1035C000C07D012802D0002874D093E04C4C012526
:1035D00040342188022906D02046478803296AD032
:1035E00004292AD132E000F07FFC6088002800D155
:1035F0006580434EB07C01281AD130462030C07B14
:10360000002815D1F08EFDF733FA31468031096A72
:1036100001F0C6FC0121C90588420FDBFDF7E4F982
:103620000006000E608009D0092801D909206080B9
:10363000B07D002804D0012805D05BE06580F7E765
:1036400000F0EAFB56E000F003FC53E02C48808ECB
:10365000FDF70EFA2A49C96C01F0AEFC284906466E
:1036600088640846807C012808D00846BF210906E6
:103670008E4229D3017C002920D020E0204F304603
:10368000FDF7B2F9BF21090660808E4203D3002006
:103690006080BD77D4E73F2109068E42D0DB002150
:1036A0000006B977000E608006D00928C8D9092025
:1036B0006080C5E71CE015E06580C1E7077385778A
:1036C000002161800574BBE73F2109068E42B7DB0C
:1036D000017B002900D10573017B61800021017409
:1036E0008177ADE7002F00D1658000F0FDFBA7E7F3
:1036F00000F0ECFB034902480968C06D8863F8BD1F
:103700000C00002030080020F8B501461F4A0024B4
:103710000B39914237D21D491D4A6A31091A50436B
:10372000FCF7DAFDFDF7A4F906461A4D02E0641C29
:10373000722C07DAA0002858314601F005FCF6D3B8
:10374000722C00DB7124A4002F593046394601F059
:1037500033FC064660198038C16F384601F02CFCF6
:1037600005460D48211804598039C96F204601F0DB
:1037700023FC2946FDF762F8314601F08DFB214616
:1037800001F044FBF8BD0548F8BD0000950F0000AE
:1037900010270000C802002000010020000020C205
:1037A00070B5344901250B88084609224038042B9E
:1037B00004D0022B08D0032B10D017E0047B092C77
:1037C00000D90273047B10E00478002C04D0092C8B
:1037D00000D90270047808E00570FBE78479002CBA
:1037E00043D0092C00D9827184794C80C67D002495
:1037F000012E00D9C4754E88002E38D0092E00D96C
:103800004A80C68E1925232E01D80F2E00D2C586D8
:10381000868E232E01D80F2E00D285860325022BFB
:1038200001D3042B00D90D80038FA021642B00D27B
:103830000187838F642B00D28187418F642901D255
:10384000B4214187017D022901D3C82900D902751D
:10385000017A012900D90472417A012900D9447200
:10386000817A012900D9847270BD8571BCE74D80D1
:10387000C7E700004C000020F0B53E4F3E4D3846F3
:1038800080383E6A43783D4C3D49827BAE4201D848
:10389000A64209DD066E8E4201D2761C06668E4275
:1038A00004D1D60714D015E000260666042B02D2F8
:1038B0005208520082732F4A566A803A526E531C45
:1038C000A6420DDC2B4F403F3F88042F05D038E047
:1038D0005B1C437001231A43ECE72A4FBE4230DAE7
:1038E0008A4200D24366426E8A422CD1214B827BAF
:1038F000803B9B7897075B1CDBB2002F01DA170730
:1039000000D4837002231A438273AE4202D9082383
:103910001A438273174A936A803AD278AB4201D82D
:10392000A34214DD836E8B4201D25B1C83668B4203
:103930000FD1817B4B0701D4521CC270042211436A
:103940000CE000224266827BF5231A40E1E7002169
:103950008166042A03D2817BFB22114081730179A5
:103960000129817B03D0EF2211408173F0BD102229
:103970001143FAE78C0000200000A0C10000F042D3
:103980008813000000003442F8B5214C0025E07D8A
:10399000012802D0002838D0F8BD1D4840300088EA
:1039A000022804D0032830D00428F5D12DE018488F
:1039B0002030007C012828D0E08EFCF712FF002286
:1039C000144BFCF7B5FE064611480F468030006ADE
:1039D000FCF70AFF32463B4601F0E4F902D201202F
:1039E0006074F8BDE08EFCF7FCFE0022094BFCF78A
:1039F000ACFE064606480F468030006AFCF7F4FE2F
:103A000032463B4601F09CF9EBD86574F8BD0000E6
:103A10000C0000200000E03FFEB5814C0026A07B9A
:103A20000A2804D2204620384676803046607D48F9
:103A300047793807000FFDF71BF87B49FCF7FEFEBE
:103A4000054678480079FDF713F8294601F0DEF9BC
:103A5000734D60353909754FE86201D07840E862EE
:103A60007048C17901910807000FFDF701F86E4910
:103A7000FCF7E4FE00906B488079FCF7F9FF0099B1
:103A800001F0C4F928630199090901D0784028633D
:103A90006448417A01910807000FFCF7E9FF624989
:103AA000FCF7CCFE00905F48007AFCF7E1FF00993C
:103AB00001F0ACF968630199090901D078406863A5
:103AC0005848C17A01910807000FFCF7D1FF564909
:103AD000FCF7B4FE00905348807AFCF7C9FF0099C8
:103AE00001F094F94E49603188630199090903D0C6
:103AF0004B496031784088634A4D687B0007000F6E
:103B0000FCF7B6FF4849FCF799FE0090287BFCF7CC
:103B1000AFFF009901F07AF941496031C863A87B91
:103B20002070E87B6070287CA0700C46687C803C2C
:103B3000A075A87CE073E87C0A214843297D4118E0
:103B4000204680308165687D0A214843A97D401860
:103B5000FCF78EFF214680310864E87D6075697E40
:103B600001910807000FFCF783FF2F49FCF766FE61
:103B70000090287EFCF77CFF009901F047F9206552
:103B80000199090901D078402065A87E6077E87E18
:103B9000E074287F6071687FE071012835D1A87FCB
:103BA0002070E87FE0861F481D49203002782031D0
:103BB0000A804178E1758178A174C1782175017915
:103BC000E17241790A224900616781795143C279E2
:103BD00089182187017A0A225143427A8918A187DC
:103BE000817A0A225143C27A89186187017B217345
:103BF000417BA186817BA171C17B2172017C6172B5
:103C0000407CA072A665FFF7CBFD064930466439BB
:103C100026678855761C322EFBD32667FEBD000032
:103C20002C000020480700200000204100000080F8
:103C3000F8B5774C01214903206D764D4F100026D1
:103C400000281BD001287BD000222846FDF75BFF0F
:103C5000002239462846FDF756FF0022012128465A
:103C6000FDF751FF092000228021C006FDF74BFF20
:103C7000E16CA06D884277DA2665F8BDE06C00281B
:103C8000F6DBA06C0300FFF707FC07050B232934C4
:103C90003F411F0001222846FDF735FF002204E0C6
:103CA00001222846FDF72FFF012239462846FDF75D
:103CB0002AFF002201212846FDF725FF00220920C6
:103CC0008021C006FDF71FFF206D00282FD034E0B3
:103CD00000222846FDF717FF012204E000222846B3
:103CE000FDF711FF002239462846FDF70CFF01229F
:103CF000E0E700222846FDF706FF00223946284665
:103D0000FDF701FF01220BE0002200E0012228461E
:103D1000FDF7F9FE002239462846FDF7F4FE0022A1
:103D200001212846FDF7EFFE0122C8E708E0A06C5C
:103D3000401EA06401D50620A064E06C401E30E067
:103D4000FF22E06C2D32904292DCA06C0300FFF762
:103D5000A3FB07050C2A303B4648200001222846D9
:103D6000FDF7D1FE002205E04BE001222846FDF7D9
:103D7000CAFE012239462846FDF7C5FE0022012170
:103D80002846FDF7C0FE002209208021C006FDF76D
:103D9000BAFEA06C401CA064062800DDA664E06C9E
:103DA000401CE06464E700222846FDF7ACFE0122D7
:103DB00004E000222846FDF7A6FE002239462846E8
:103DC000FDF7A1FE0122DAE700222846FDF79BFE5F
:103DD000002239462846FDF796FE01220BE000221C
:103DE00000E001222846FDF78EFE002239462846D3
:103DF000FDF789FE002201212846FDF784FE0122FD
:103E0000C2E7884201DD012000E002202065F8BD04
:103E10008C0000200004004810B50C484188403850
:103E200000290DD0428F038F491ED21AD417640F78
:103E3000A218D2104A43C16DD2188A4202D9491C35
:103E4000C16510BD8A42FCD2491EF9E74C00002032
:103E50000B48418F828F891ACB175B0F5918034685
:103E600040335B88C9105B1E59438A18C16D8A4272
:103E700001D9491C02E08A4201D2491EC16570473E
:103E80000C00002070B50E4C0025E06D642815D99B
:103E90000121C9030B48FDF72BFE012801D0656401
:103EA0000AE00949606C884201DA401C606488427B
:103EB00002DB0120207170BD257170BD656470BD8D
:103EC0000C00002000040048204E00000548028F2E
:103ED000C16D0A3A914201D9491E00E00021C16535
:103EE000704700000C0000200348018FC26D0A39A2
:103EF0008A4200D2C16570470C0000200EB5FDF764
:103F000017FEFEF7ADFEC820FDF79AFCFEF782FD16
:103F1000FEF774FDFEF72AFDFEF7F0FDFEF75AFEF0
:103F2000FEF774FE7D25ED002846FDF789FCBD4CAB
:103F3000012211462046FDF7E6FD0122BA4F960305
:103F400031463846FDF7DFFDB848FDF7BFF9284692
:103F5000FDF776FC0322B649B448FDF79DFB2846E1
:103F6000FDF76EFCFDF70CFDFCF7B8FF2846FDF7EA
:103F700067FC00F015FA2846FDF762FC0122AD4906
:103F8000AD48FEF739FC2846FDF75AFCA949012245
:103F9000491EAA48FEF730FC2846FDF751FCA84808
:103FA0000025006885630421A548FEF799F90022E1
:103FB00001212046FDF7A7FD002231463846FDF7D6
:103FC000A2FD9C4CFF27323C204640302567264608
:103FD000C33720360090FFF72BFE1420FDF730FC8E
:103FE000206F401C2067B842F5D3607EA17B084358
:103FF00006D00120707393480178012907D074E03E
:104000007573002201218748FDF77DFDF3E70570F8
:10401000E06E884F401CE066E06F4E37401CE06762
:104020003868401C3860786C401C7864FA2807D1E6
:104030007D64707B012803D101217A48FDF75DFD85
:10404000786D401C7865142802D17D65FFF7F0FD7E
:10405000606D401C6065642802D16565FFF7AEFAAB
:104060007949A06D884202D2401CA06505E08842D3
:1040700003D1401CA06500F0BFFD7D21A06FC900E9
:10408000884201D2401CA06770497868884201DAF2
:10409000401C7860884207D1607E002802D1B07B46
:1040A000401CB073012060764B213868C9008842FB
:1040B00002D13D6000F0CCFCFF27E06EF537B8423E
:1040C00005D1012189035848E566FDF716FDE06F2B
:1040D000B84202D1E56700F005FB00F0BDF8FFF73C
:1040E000CBFBFFF709FAFFF7CDFEA07E01287DD1BB
:1040F000A57600F031FAB079012877D1544FB57127
:10410000F878102802D020285FD074E03879207326
:104110000290787920708446B879A0710190F8797E
:10412000E0860099387A0880797AE1752346B97A71
:104130009974F97A1975397BD972797B0A22490009
:104140005967B97B1977F97B51433A7C89181987EC
:10415000797C0A225143BA7C89189987F97C0A2212
:1041600051433A7D89185987797D9986B97D1972AD
:10417000F97D5972397E9972042804D0022809D039
:10418000032812D01BE00298092801D909201873CE
:10419000197B12E06046002805D0092801D90920C2
:1041A0001870C1B209E00120FAE7019800280AD08E
:1041B000092801D909209871997900984180A5654D
:1041C000FFF7EEFA17E00120F5E77879FCF750FCED
:1041D0002049FCF733FB01903879FCF749FC019941
:1041E00000F014FEE064B979012900E00AE002D190
:1041F000C9074840E064284625673D54401C3228E2
:10420000FBD32067E07E012808D1E57600F00CFAA8
:10421000F07A012802D1F572FFF7FEFBFFF7B4FB3D
:10422000E3E600000014004800080048AC07002046
:10423000380500203E00002070080020F008002013
:1042400030080020FC040020881300001027000024
:10425000E406002000002041F8B54E4CFF27A06E78
:10426000F537B8420EDA4C49E36D0A68D218E265B8
:104270004A68236ED21822668968626E8918401CCB
:10428000616684E0B8427DD13946E06DFCF724F8E0
:10429000404D424A803DE97F8E00905109CA116825
:1042A000C01840180321FCF717F83C4A0C32905113
:1042B00009CA1168C01840180321FCF70DF83749E6
:1042C0001831885105C90968801840180321FCF786
:1042D00003F8FFF719FA60623946206EFBF7FCFF1E
:1042E000E97F2E4A8E00243A905109CA1168C018FD
:1042F00040180321FBF7F0FF284A183A905109CAE9
:104300001168C01840180321FBF7E6FF23490C3958
:10431000885105C90968801840180321FBF7DCFFA4
:10432000FFF7F2F920623946606EFBF7D5FFE97FAF
:104330008E001A492431885105C90968801840182F
:104340000321FBF7C9FF15493031885105C90968B8
:10435000801840180321FBF7BFFF10493C318851FA
:1043600005C90968801840180321FBF7B5FFFFF75E
:10437000CBF9A062E87F401CC1B20020E977032995
:1043800002D100E004E0E877E06520666066A066A0
:10439000F8BD00008C00002038050020B404002087
:1043A000F0B56B4C89B0A11C6520FCF7A9FE642018
:1043B000FDF746FA211D6620FCF7A2FE6420FDF7FA
:1043C0003FFAA11D6720FCF79BFE6420FDF738FA39
:1043D000214608316820FCF793FE6420FDF730FA8F
:1043E00021460A316920FCF78BFE6420FDF728FA8C
:1043F00021460C316A20FCF783FE6420FDF720FA89
:1044000021460E316B20FCF77BFE6420FDF718FA85
:10441000214610316C20FCF773FE6420FDF710FA82
:10442000214612316D20FCF76BFE6420FDF708FA7F
:10443000214614316E20FCF763FE6420FDF700FA7C
:10444000214616316F20FCF75BFE6420FDF7F8F97A
:10445000214618317020FCF753FE6420FDF7F0F977
:1044600021461A317120FCF74BFE6420FDF7E8F974
:1044700021461C317220FCF743FE6420FDF7E0F971
:1044800021461E317320FCF73BFE6420FDF7D8F96E
:10449000214620317420FCF733FE6420FDF7D0F96B
:1044A000214622317520FCF72BFEA0880890E18878
:1044B000079142182089618986464018A6898C4652
:1044C00010188119E08906900918208A05900918AA
:1044D000608A04900918A08A03900918E08A029063
:1044E0000918208B0190658B08184119A08B00904A
:1044F0000818E38B228CC018618C80184018C043C8
:10450000144F80B2F887648884421CD1089CFC86D2
:1045100038464037079C3C807446C4756446047531
:10452000C672069C0477059C0487049C8487039CC0
:104530004487029C0473019C04708571009C8486EE
:10454000037242728172FFF72BF909B0F0BD0000CF
:10455000100500200C000020F0B53148314B0278E6
:104560001238C17802255A541E78491C0479002259
:10457000C9B25A2E08D0002C0ED0012C09D0022C22
:1045800012D0032C1DD01DE0002CF6D1C1700121EA
:1045900015E05C78A52C02D0C270027112E0C170E7
:1045A00002290FD905710DE09C78241DE4B24471F5
:1045B000641E5F2C30D2C170032903D9032101711D
:1045C00000E0C170C1784479A14228D10179032962
:1045D00025D113494E318A61C5711146661E03E02B
:1045E0005F5D79186D1CC571EDB2B542F8DB0C4DFD
:1045F000C9B24E351C19203CA961E47F8C4202D11E
:104600000121817108E0064C1146323C22675A5460
:10461000491C3229FBD32167C27002714271F0BD7F
:104620003E000020E4060020F0B52C482C4B027818
:104630001138017A02265A54491C1D78CAB2447AAC
:1046400000215A2D08D0002C0ED0012C09D0022CAC
:1046500012D0032C1DD01DE0002CF6D102720122D5
:1046600015E05C78A52C02D00172417212E0027252
:10467000022A0FD946720DE09C78241DE4B28472A0
:10468000641E5F2C26D20272032A03D903224272CF
:1046900000E00272027A857AAA421ED1427A032A87
:1046A0001BD10E4A0C464F32D16106736E1E03E0D9
:1046B0009F5C3C19521C0273027BB242F8DB074A32
:1046C000E4B24F32D4615A19203AD27FA24201D1CA
:1046D0000122C272017241728172F0BD3D00002060
:1046E00048070020F8B5D24D10206870D14C022048
:1046F000A060D14EE06AD14FB04208D2394600F0F6
:10470000CBFBFCF74BF90A21FBF7F0FD08E0CC49A5
:1047100000F0C2FBFCF742F90A21FBF7E7FDF0319C
:1047200061612061207CA870207DE8700420A06079
:10473000206BB04208D2394600F0AEFBFCF72EF9F0
:104740000A21FBF7D3FD08E0BD4900F0A5FBFCF70B
:1047500025F90A21FBF7CAFDF03161612061207C57
:104760002871207D68710620A060606BB04208D27D
:10477000394600F091FBFCF711F90A21FBF7B6FD71
:1047800008E0AF4900F088FBFCF708F90A21FBF7C5
:10479000ADFDF03161612061207CA871207DE87160
:1047A0000820A060A06BB04208D2394600F074FB2C
:1047B000FCF7F4F80A21FBF799FD08E0A04900F0A6
:1047C0006BFBFCF7EBF80A21FBF790FDF031616120
:1047D0002061207C2872207D68729849E06B00F08F
:1047E0005BFBFCF7DBF80A21FBF780FD61612061D0
:1047F000904FA872E972603F3878287378786873B0
:10480000B878A8730F20A060206AB04208D28B4904
:1048100000F042FBFCF7C2F80A21FBF767FD08E055
:10482000874900F039FBFCF7B9F80A21FBF75EFD78
:10483000F03161612061207CE873207D28741120B3
:10484000A060606AB04208D27C4900F025FBFCF70A
:10485000A5F80A21FBF74AFD08E0794900F01CFBA6
:10486000FCF79CF80A21FBF741FDF0316161206102
:10487000207C6874207DA8741320A060FF21A06AAA
:10488000C905C84208D26D4900F006FBFCF786F85E
:104890000A21FBF72BFD08E0694900F0FDFAFCF75F
:1048A0007DF80A21FBF722FDF03161612061207C57
:1048B000E874604E207D2875803E707E6875307E7D
:1048C000A875307BE87530782876B0796876F08EF8
:1048D000A876304640300078E876F07D2877B07DC5
:1048E0006877B07BA877F07BE8772020317D29546A
:1048F000A06D2122C10F08184010A854206CFCF7AD
:104900004DF80A21FBF7F2FC2222A8542320295457
:104910002421707D68542520A0600090FF21306D17
:10492000C905C8420DD2474900F0B6FAFCF736F87F
:104930006421FBF7DBFC61612061009800212954B0
:104940000CE0414900F0A8FAFCF728F86421FBF7D5
:10495000CDFC616120610099012068542620A0608F
:10496000A168207C68542720217D29542820717F4C
:104970002954F07C292168540A21308FFBF7ACFCC4
:104980002A22A8542B2029540A21B08FFBF7A4FC1B
:104990002C22A8542D2029540A21708FFBF79CFC4F
:1049A0002E22A8542F202954302031792954312027
:1049B000717929543220F97B29543320B17F29544D
:1049C0003421B08E68543520317A29543620717ADA
:1049D00029543721B07A6854A16015480A462970D5
:1049E0005A21C8300170A5214170372181703730BC
:1049F000C17001203067501C316F0AE00C4B6C5CB9
:104A0000C8335F18BC709B18DF783C19DC70491CF8
:104A100031678142F2D306490C48C831121DFDF7B7
:104A200067FF044901224E390848FDF7E5FEF8BD4D
:104A3000540500208C0000200000808000002041F0
:104A4000000020C10000C8420000C8C27008002059
:104A5000F8B5634F10207870624C0220E060624D20
:104A6000206A624EA84208D2314600F015FAFBF7E0
:104A700095FF0A21FBF73AFC08E05D4900F00CFACB
:104A8000FBF78CFF0A21FBF731FCF03161612061FB
:104A9000207CB870207DF8700420E060606AA84235
:104AA00008D2314600F0F8F9FBF778FF0A21FBF74E
:104AB0001DFC08E04E4900F0EFF9FBF76FFF0A21FB
:104AC000FBF714FCF03161612061207C3871207D9E
:104AD00078710620E060A06AA84208D2314600F052
:104AE000DBF9FBF75BFF0A21FBF700FC08E040491C
:104AF00000F0D2F9FBF752FF0A21FBF7F7FBF03188
:104B000061612061207CB871364D207DF871803D57
:104B1000687C3872A87B78722878B872E88EF87250
:104B20002846403000783873E87D7873287DB87364
:104B3000E87AF873E06CC10F081840103874686F99
:104B4000C10F081840107874287FB8740A21288F84
:104B5000FBF7C2FBF87439750A21A88FFBF7BCFB81
:104B60007875B9750A21688FFBF7B6FBF875397649
:104B7000287B7876A88EB876A879F876287A387760
:104B8000687A7877A87AB8771E221548E2603A707A
:104B90005A21C8300170A521417082701E30C27048
:104BA00001202B462867511C186F0AE00C4C3D5C15
:104BB000C8342618B570A418E6787519E570401C3D
:104BC00018678842F2D306490A48C831121DFDF71A
:104BD0008FFE044901224F390648FDF70DFEF8BD4E
:104BE000B80500208C0000200000808000002041DB
:104BF000000020C1F0080020F0B5012291B011465C
:104C00004C48FCF780FFFEF7CBFD4B484B4CC78E62
:104C10000146A78040310A88E280C17D2181037D61
:104C200063810093C37AA3810F93037FE3810E9383
:104C3000038F23820D93838F63820C93468FA6820A
:104C4000057BE582037823839E46837963830893FB
:104C5000838EA3830793037AE3830693437A2384A3
:104C60009C46837A6384BF18009A89187A180F9932
:104C700052180E9952180D9952180C9951188919F9
:104C80004A190899724452180799521806995218ED
:104C900061465118C918C94389B2C187618065202E
:104CA000FCF78EFAA1886620FCF78AFAE188672073
:104CB000FCF786FA21896820FCF782FA618969206D
:104CC000FCF77EFAA1896A20FCF77AFAE1896B2069
:104CD000FCF776FA218A6C20FCF772FA618A6D2063
:104CE000FCF76EFAA18A6E20FCF76AFAE18A6F205F
:104CF000FCF766FA218B7020FCF762FA618B712059
:104D0000FCF75EFAA18B7220FCF75AFAE18B732054
:104D1000FCF756FA218C7420FCF752FA618C75204E
:104D2000FCF74EFA002201210248FCF7ECFE11B01C
:104D3000F0BD0000001400480C0000201005002009
:104D400070B501250C002D051C4310D4EC4206D48F
:104D5000AC420AD4994200D070BD904270BDE94285
:104D600017D4EB4215D4994270BD894270BDEC4214
:104D700006D5AC42F9D58B4200D070BD824270BDE1
:104D80006D004C00EC4204D25C00EC4201D28B423C
:104D900070BD034C30B4FBF76FFE30BC70BD00BF7C
:104DA0001900160470B501251C002D050C4310D404
:104DB000EC4206D4AC420AD48B4200D070BD824291
:104DC00070BDEB4217D4E94215D48B4270BD9B42B3
:104DD00070BDEC4206D5AC42F9D5994200D070BD09
:104DE000904270BD6D005C00EC4204D24C00EC427D
:104DF00001D2994270BD0FB4034C0CBC03BC30B45B
:104E0000FBF73AFE30BC70BD1900160470B50125E1
:104E10000400ED074C4020D4441A01D2001B0919AC
:104E2000C60D4B00F2B2FF2A29D01B0E2CD0000277
:104E30000C02D31A2C43DC402843051910D2280A4F
:104E400002D3401C6D0611D0761EF6058019FF2A8C
:104E500000DA70BDC00DC00570BD694000F0B2F849
:104E600001200543C541521C761CE8E764089C40BC
:104E7000C90161408900E7D10124A043E4E71B0E8A
:104E8000440200D0034870BD002AFCD1C00FC00707
:104E900070BD00BF0000C07F70B5420064414B0090
:104EA0005C41120E39D01B0E38D0FF2A3CD0FF2BAC
:104EB0003AD040024902400A490A060045184E43CA
:104EC000000A090AD2184843ED017F3A0104731A17
:104ED0004019190C4318990F04D001215B084907A8
:104EE0005B1A521CD80904D3401CF50301D19D065E
:104EF00007D0FF2A08D2D50506D0E4072043401981
:104F000070BD0125A843F4E7002A01DCE00770BD6D
:104F10002402FF202043C00570BD1B0EFF2A03D0D2
:104F2000FF2B01D0E00770BDFF2645003606B542D5
:104F300006D84D00B54203D8D218FF2A00D0E7E7C3
:104F4000004870BD0000C07F01230A00DB0502435A
:104F50000DD4DA4203D49A4207D481427047D94231
:104F600014D4D84212D48142704789427047DA4241
:104F700003D59A42F9D5884270475B004A00DA426D
:104F800004D24200DA4201D2884270474840414090
:104F900010B5024A4840FBF7B7FD10BD09001604E2
:104FA00070B50125ED07684004004C4002D569400A
:104FB00000F008F8FFF730FF70B501250400ED0799
:104FC0004C4022D4441A02D26C40001B0919C60D71
:104FD0004B00F2B2FF2A4BD01B0E50D000020C0245
:104FE000D31A2C43DC40A843051B05D5AD0019D3CB
:104FF0006D08761E521E37D0F605280A01D2801998
:1050000070BD70416D0603D070BD6940FFF704FFAD
:105010009C4009026140490001D0401E70BD01243E
:10502000A04370BD6D081DD001202B0C01D12D04B3
:1050300010302B0E01D12D0208302B0F01D12D0184
:10504000001DAB0F01D1AD00801CEB0F01D16D0035
:10505000401C6D00361A121A680AF5054019012A1B
:1050600002DB70BD002070BDC036300AC00770BDC5
:105070001B0E440201D1FF2B00D1024870BD002A53
:10508000F0D070BD0000C07F0000000000000000F4
:1050900001020304060708090000000001020304DE
:1050A0008182838485868788898B8C8D8E8F91926F
:1050B00093959697999A9C9D9FA0A2A3A5A7A8AA0D
:1050C000ACAEB0B2B3B5B7B9BCBEC0C2C5C7C9CC2F
:1050D000CED1D4D7D9DCDFE2E6E9ECF0F3F7FAFE83
:1050E000005100080000002010050000820C00089C
:1050F0006854000810050020E00A0000F8000008CD
:1051000001230220011264145E0164023D0532078E
:105110003203051A48F4FFFF0B1820C20431754012
:105120009C45C80A1FC1B66118108FC21DC2EC5140
:1051300019C248E114C2A470104820230CC25C8F2D
:1051400007C2B81E03C2295CFDC1E17AF4C11F8504
:10515000EBC1D7A3E2C18FC2D9C148E1D0C1180EBB
:10516000C8C1B81EBFC1713DB6C1295CAD241AA427
:10517000241A9B241A92241A89241A80241A702033
:105180001A5E1C18124CC152B83AC1C3F528C13D71
:105190000A17C1AE47050827E7C01F85C3C02812FC
:1051A000A0C0C3F578C085EB31C08FC2D5BF295CE4
:1051B0000F041A3F0C1A3F141A401C1A40241A40BC
:1051C0002C1A40341A403C1A41441A414C1A41549A
:1051D0001A415C1A41641A416C1A41741A417C1AD2
:1051E00041841A418C191C1BA4419C19201BB641F7
:1051F000AC19241AC8241AD0241AD9241AE2241A61
:10520000EB241AF4241AFD201B0342F41A42FC1862
:105210001D42A470104248E11442EC5119428FC261
:105220001D42713D224214AE2642B81E2B241A2F75
:10523000241A34241A38241A3C241A41241A4524E6
:105240001A4A241A4E241A53241A57241A5C241A70
:1052500060241A64241A69241A6D241A72241A7696
:10526000241A7B241A7F241E8242523884281E86E8
:1052700042F6A8882C1A8A1C1E8D420A578F201EBF
:105280009142AEC793241A96241A98241A9A241A83
:105290009C241A9E241AA1241AA3241AA5241AA70E
:1052A000241AAA24100BAC42E01F9E48C0F5924875
:1052B0001018A98848804E7E48C0BE6C4840845C67
:1052C00048C0824D48C0A03F481008C73248C0C5FA
:1052D000264814C01B4814881148140D08481010A3
:1052E00081FE478029EE4780FADE4780DDD04710F7
:1052F00008BDC347806AB747140DAC471477A14770
:1053000010089A974780678E4714D3854714A37B6C
:105310004714B06C4714B95E47148F5147145E456B
:105320004714F63947144A2F47144D254714F11BEB
:1053300047142C134714F50A47143F034714E8F7A2
:10534000461458EA46149ADD4614A4D1461466C69B
:105350004614D4BB4614E4B146148AA84614BC9F34
:10536000461460974614948F46143A8846144C812C
:1053700046148875461434694614905D4614985254
:10538000461B384844133E461B183508132C461458
:1053900014244614401C461BD814041A0D2C130761
:1053A0004612EC124614D0F5451488EA4514D8DFAD
:1053B0004514B0D5451410CC4514F0C2451440BA7C
:1053C000451408B2451438AA4514B8A2451BA89B39
:1053D000181A942C138E451B78882C138245146060
:1053E0007A451BE06F181365451B505C3413534519
:1053F00014A04A45147042451B903A4C1A331C13B2
:105400002B451B2025181A1E301A181C1312451B79
:10541000C00C301A07181A021413FA441BE0F004E7
:1054200013E7441420DF441BC0D60C13CE442440A1
:10543000C7441AC00413B9441B60B2141AAB1C1A37
:10544000A5081A9F1C1A9A0C1394441BA08F041AC7
:105450008A0C1A8514258144D0070966044132015B
:08546000820413127A0000001F
:04000005080000B53A
:00000001FF
